:020000040000FA
:06000000A0EF3EF000003D
:0C7D34009AEF3EF0000000009CEF3EF0D3
:107D4000D0A69CEF3EF0900EAB6EAC84AC8A330EA6
:107D5000AF6E070EC16E8B90949080BAD9EF3EF053
:107D60008D8296928B9A949A8D949694898089822A
:107D700092909292BCEF3EF030EC3FF0756EE30AC9
:107D8000D8B4E6EF3EF07550E60AD8B4E6EF3EF020
:107D90007550EA0AD8B4DFEF3EF07550ED0AD8A46A
:107DA000BCEF3EF0E40E2AEC3FF00B0E736E30ECAD
:107DB0003FF0CD6AAB6AAC6A9E6A9CEF3EF079EC0C
:107DC0003FF08AEC3FF0EB0E26EF3FF030EC3FF057
:107DD000006E30EC3FF0016E070B766E00EE20F087
:107DE00006E0FF0EEE6E01060150070BF9D730ECEE
:107DF0003FF0776E7742746E30EC3FF0726E716ACE
:107E000030EC3FF0786E712630EC3FF0EE6E71266C
:107E100078C0EEFF7706F4E171507218E80ED8A42E
:107E200015D0E70E2AEC3FF0765074267450070BFD
:107E300004E0FF0EEE6E742AF9D774427442744265
:107E400036EC3FF00009E40ED8B4E50E2AEC3FF022
:107E5000BCEF3EF004009EA82AEF3FF0AD6E12008A
:107E600004009EAA30EF3FF0AE5012007550E60AB3
:107E7000D8B433D07550E30AD8A4000C005029E1DF
:107E8000040E015C26E27D0E006E380E016E10EECF
:107E900020F000EE40F0FF0E776EE7CFEEFFE750E8
:107EA00077C0E6FFEF0AF9E1E7CFEEFFFF0EE66EDF
:107EB000E7CFEEFFEE6EEE6EEE6EEE6E74C002F089
:107EC000010E746E00EE40F00BD8016A006A02C029
:107ED00074F000EE20F004D8010C21C0F8FF010C72
:107EE00000C0F7FF01C0F6FFD7EC3FF07406FCE1DD
:107EF0001200F86AF76AF66A21EEF5F0040066D817
:107F0000400EF626D8B0F72ADD52D952F7E1DA5200
:107F1000F5E1120000EE20F0000E7B6ED8907B326F
:107F2000F00E7B127D0E7A6E7A32400E786E7832C9
:107F3000EF0E796E10EE78F0040E746EE6CFEEFF61
:107F40007406FCE1FF0EEE6EEE6EEE6EEE6EF66AFD
:107F5000F76AF86A00EE20F0D7EC3FF0000E7B6E77
:107F6000D8907B32F00E7B127D0E7A6E7A32340E10
:107F7000786E7832EF0E796E00EE20F0FF0EEE6E26
:107F8000EE6EEE6EEE6E10EE78F0040E746EE6CFCE
:107F9000EEFF7406FCE1000EF86E7D0EF76E340EF7
:107FA000F80BF66E00EE20F0D7EC3FF01200080E52
:107FB0000A6EEECFF5FF0D000A06FBE10A00A68E61
:107FC000A684ECEC3FF0A69409001200A68EA684CD
:107FD000A688ECEC3FF01200550EA76EAA0EA76E15
:067FE000A6820000120061
:020000040030CA
:0E000000FFFEFCFEFFFFFBFFFFFFFFFFFFFF09
:00000001FF
